:03000000020026D5
:050003007F05DFFE2275
:03000B0002018D62
:0D000E00C2C1D2C0120003D2C112000322F1
:030023000201D601
:10002600758123E4787FF6D8FD9005FBE493700292
:10003600804EC31392D5C31392D1FFA3E493F8B0B5
:10004600D5402130D505E4A393F5A0E420D102A341
:100056009320D507F608DFF3A380D1F208B800F69F
:1000660005A080F2E8030303541F2420F9E854078F
:10007600F8E4D333B80002800333D8FD47F780D8BD
:0600860075A0FF0205E574
:10008C008F221201581201467F901201157F4012E7
:0B009C000115AF2212011512000E2208
:1000A7008F1D1201581201467F90120115E51D544C
:1000B700034440FF12011512000E1201467F9112F0
:1000C7000115D2021200DBC2021200DB8F1E1200E2
:0400D7000EAF1E2228
:0500DB00D2C1752108EF
:1000E000D2C0120003A2C192E723120003C2C012C1
:0A00F0000003D521EBAEE03002045E
:0400FA00C2C18002FD
:1000FE00D2C1120003D2C0120003C2C0120003C24A
:07010E00C11200038E07225D
:050115008FE0751F08DA
:10011A00A2E792C1120003D2C023120003C2C01286
:10012A000003D51FEBD2C1120003D2C0120003A2F2
:0C013A00C19201120003C2C01200032297
:10014600D2C1D2C0120003C2C1120003C2C0120043
:02015600032282
:0B015800D2C1120003D2C0120003222B
:10016300758F034387C07598528F9A759B1EC299EA
:07017300C298D2BCD2AC22FD
:10017A005389F0438902758C80758A80C28DC28C3E
:03018A00D2A922D5
:0F018D00C0E0C0D0C002C003C007E508F4700C8A
:0C019C00E5A054F0FFE5094FF5A080231A
:0301A80020001123
:1001AB0085088CD200E5A054F0FFE5094FF5A0803F
:0101BB000F34
:1001BC0074FFC39508F58CC200E5A054F0F5A0D0EF
:0A01CC0007D003D002D0D0D0E032FB
:1001D600C0E0C0F0C083C082C0D0C000C001C00271
:0E01E600C003C004C005C006C007C2AC7F0045
:1001F4003098FDEF2410F8A699C2980FBF03F1E5DB
:1002040010B406030202E05014E51014602E1460CA
:100214003514603F146046146050020479E51024DC
:10022400F9700302033524FD700302045E147003A5
:0C02340002046514700302046F020479D8
:10024000AF11AD12120498020479AF111204AD8FF0
:10025000993099FD020479AF11AD121205830204A1
:1002600079AF111200A78F993099FD02047912011C
:10027000581201467FC01201157F021201151201AA
:10028000467FC1120115E4F513751430E513B4006F
:1002900006E514B40001D3400AE514151470ED15F9
:1002A0001380E9D2021200DB8F15851599C2021264
:1002B00000DB8F1612000E3099FD7513087514FFC0
:1002C000E513B40006E514B40001D3400AE51415A3
:1002D0001470ED151380E98516993099FD020479A3
:1002E0001201581201467FC0120115E4F51375146E
:1002F00020E513B40006E514B40001D3400AE51468
:10030000151470ED151380E97F0F120115E4F51334
:10031000751420E513B40006E514B40001D3400AB7
:10032000E514151470ED151380E9AF1112011512C3
:10033000000E0204791201581201467FA412011521
:100340007FF01201157F5512011512000E120146A1
:100350007FA41201157FFB120115E4FF1201151293
:10036000000E1201467FA4120115E4FF12011512BE
:10037000000E1201467FA5120115D2021200DB8F7A
:1003800017D2021200DB8F18D2021200DB8F19D2B3
:10039000021200DB8F1AD2021200DB8F1BC2021284
:1003A00000DB8F1C12000E8517993099FD75130F15
:1003B0007514FFE513B40006E514B40001D3400A38
:1003C000E514151470ED151380E98518993099FD21
:1003D00075130F7514FFE513B40006E514B400019E
:1003E000D3400AE514151470ED151380E9851999A9
:1003F0003099FD75130F7514FFE513B40006E5146D
:10040000B40001D3400AE514151470ED151380E90A
:0C041000851A993099FD75130F7514FFC3
:10041C00E513B40006E514B40001D3400AE5141545
:10042C001470ED151380E9851B993099FD75130F28
:10043C007514FFE513B40006E514B40001D3400AAB
:10044C00E514151470ED151380E9851C993099FD90
:10045C00801BAF1112008C8014E590F4F599309943
:10046C00FD800AE5116004D2A48002C2A4C299D214
:10047C00ACD007D006D005D004D003D002D001D028
:0C048C0000D0D0D082D083D0F0D0E0327D
:100498008F098D0853A0F0E50942A0E5097003C251
:0504A8008C22D28C2221
:1004AD00EFBF10004003020580FE232F9004BD73A3
:1004BD000204F00204F902050202050B0205140202
:1004CD00051D02052602052F02053802054102050C
:1004DD004A02055302055C02056502056E020577A9
:0304ED0002058085
:1004F0003090037F0122E4FF223091037F0122E448
:10050000FF223092037F0122E4FF223093037F0118
:1005100022E4FF223094037F0122E4FF223095037E
:100520007F0122E4FF223096037F0122E4FF223084
:1005300097037F0122E4FF2230A4037F0122E4FF1E
:100540002230A5037F0122E4FF2230B2037F012283
:10055000E4FF2230B3037F0122E4FF2230B4037FA3
:100560000122E4FF2230B5037F0122E4FF2230B6EE
:10057000037F0122E4FF2230B7037F0122E4FF2240
:03058000E4FF2273
:10058300BF0C02803D500FEF24F8601614601B145B
:10059300602014602522EF24F3602F14603414606C
:0205A3003922FB
:1005A500EDFBEB24FF92A422EDFBEB24FF92A522A9
:1005B500EDFBEB24FF92B222EDFBEB24FF92B3227D
:1005C500EDFBEB24FF92B422EDFBEB24FF92B52269
:1005D500EDFBEB24FF92B622EDFBEB24FF92B72255
:0F05E50075A000AF0C12016312017AD2BCD2AF25
:0705F400E590F4F58080F9A9
:0F05FB00040BE6040CD9040DCC040EB2040F64FB
:01060A0000EF
:00000001FF
